:1000000019C018951895189518951895189518955C
:100010001895189518951895189518951895189578
:1000200017C018951895189518951895189518953E
:10003000189518950FEF0DBF02E00EBF00E004BD4C
:1000400005E005BD01E000936E0022277894FFCF04
:10005000203049F400E005B908B90BB904B907B973
:100060000AB923951895213039F40FE304B907B97B
:100070000FEF0AB9239518950FE305B908B90FEFEB
:060080000BB922271895C0
:00000001FF
